:0200000480007A
:100000006F00C004732F2034930F8000630AFF0336
:10001000930F90006306FF03930FB0006302FF038A
:10002000170F0080130F0FFE63040F0067000F000F
:10003000732F203463540F006F004000136E9E53E3
:10004000171F00002320CFFD6FF09FFF732540F1A5
:100050006310050073251030635805000F00F00F82
:10006000130E100073000000130E00009702000032
:10007000938282F973905230735020307350303035
:1000800073504030970200809382C2F7638C020065
:10009000739052109302B01A739022307323203061
:1000A000E39E62F873500030970200009382420191
:1000B00073901234732540F17300203093000000D8
:1000C00093810000930E0000130E2000639CD12743
:1000D0009300100093811000930E2000130E300047
:1000E0006392D1279300300093817000930EA0009B
:1000F000130E40006398D125930000009381008087
:10010000930E0080130E5000639ED123B700008031
:1001100093810000B70E0080130E60006394D1231A
:10012000B700008093810080B70E0080938E0E8010
:10013000130E70006398D121930000009381F07F2B
:10014000930EF07F130E8000639ED11FB7000080D6
:100150009380F0FF93810000B70E0080938EFEFF26
:10016000130E90006390D11FB70000809380F0FFC2
:100170009381F07FB70E0080938EEE7F130EA00068
:100180006392D11DB70000809381F07FB70E00808D
:10019000938EFE7F130EB0006396D11BB7000080D4
:1001A0009380F0FF93810080B7FEFF7F938EFE7FE8
:1001B000130EC0006398D119930000009381F0FFE3
:1001C000930EF0FF130ED000639ED1179300F0FF43
:1001D00093811000930E0000130EE0006394D1177A
:1001E0009300F0FF9381F0FF930EE0FF130EF000F9
:1001F000639AD115B70000809380F0FF93811000BF
:10020000B70E0080130E0001639ED1139300D0003F
:100210009380B000930E8001130E10016394D013ED
:10022000130200009300D0009381B00013830100FB
:100230001302120093022000E31652FE930E800177
:10024000130E20016310D311130200009300D0009D
:100250009381A00013000000138301001302120019
:1002600093022000E31452FE930E7001130E30012E
:10027000631AD30D130200009300D0009381900005
:10028000130000001300000013830100130212008A
:1002900093022000E31252FE930E6001130E400100
:1002A0006312D30B130200009300D0009381B000BF
:1002B0001302120093022000E31852FE930E8001F5
:1002C000130E50016390D109130200009300D00077
:1002D000130000009381A00013021200930220007B
:1002E000E31652FE930E7001130E6001639CD1055C
:1002F000130200009300D000130000001300000060
:10030000938190001302120093022000E31452FE26
:10031000930E6001130E70016396D10393000002E7
:10032000930E0002130E8001639ED0019300100211
:1003300013802003930E0000130E90016314D0016C
:10034000631CC0010F00F00F63000E00131E1E009F
:10035000136E1E00730000000F00F00F130E10004C
:1003600073000000731000C00000000000000000D7
:10037000000000000000000000000000000000007D
:040380000000000079
:1010000000000000000000000000000000000000E0
:1010100000000000000000000000000000000000D0
:1010200000000000000000000000000000000000C0
:1010300000000000000000000000000000000000B0
:081040000000000000000000A8
:040000058000200057
:00000001FF
